:100000000C9458010C9444040C9475010C947501E3
:100010000C9475010C9475010C9475010C94750188
:100020000C9475010C9475010C9475010C94750178
:100030000C9475010C9475010C9475010C94750168
:100040000C9475010C9475010C9475010C94750158
:100050000C9475010C9475010C9475010C94750148
:100060000C9475010C94750141542B4342430D0AC5
:100070000041542B43495047534D4C4F433D312C85
:10008000310D0A002B53415042523A20312C31009D
:1000900041542B53415042523D302C310D0A004106
:1000A000542B53415042523D322C310D0A004154E1
:1000B0002B53415042523D312C310D0A0041542BFB
:1000C00053415042523D332C312C22505744222C64
:1000D00022696E7465726E6574220D0A0041542B9C
:1000E00053415042523D332C312C2255534552221C
:1000F0002C22696E7465726E6574220D0A0041547B
:100100002B53415042523D332C312C2241504E2230
:100110002C22696E7465726E6574220D0A0041545A
:100120002B53415042523D332C312C22434F4E54DD
:10013000595045222C2247505253220D0A000A42A0
:100140004154544552595B6D565D3D00204C41541D
:1001500049545544453D00205554430A204C4F4EC8
:10016000475449545544453D000D0A002C000D0AE2
:1001700020687474703A2F2F6D6170732E676F6FE3
:10018000676C652E636F6D2F6D6170733F713D00FD
:1001900041542B434E45544C494748543D300D0A79
:1001A00000415426570D0A0041542B4950523D3905
:1001B0003630300D0A0041542B4353434C4B3D30F5
:1001C0000D0A0041542B4353434C4B3D320D0A0062
:1001D00041542B4346554E3D310D0A0041542B43AB
:1001E00046554E3D340D0A0041542B434C49503D79
:1001F000310D0A00220A0D0041542B434D47444162
:100200003D2244454C20414C4C220D0A0041542BC8
:10021000434D47533D220041542B434D47463D310A
:100220000D0A004154480A0D0041542B43464752E1
:10023000493D310A0D0041542B4350494E3D223176
:10024000313131220A0D00415445300A0D0041542C
:100250002B4350494E3F0A0D002B4350494E3A2044
:1002600053494D2050494E002B4350494E3A20529D
:10027000454144590041542B435245473D300A0DF6
:100280000041542B435245473F0A0D002B43524532
:10029000473A20302C35002B435245473A20302C2A
:1002A000310052494E47004F4B0041540A0D0000A7
:1002B00011241FBECFEFD8E0DEBFCDBF11E0A0E01C
:1002C000B1E0E6E8FBE002C005900D92A639B10767
:1002D000D9F711E0A6E9B1E001C01D92A33CB10736
:1002E000E1F70E944F040C94C1050C94000082E0D9
:1002F0008093C0001092C5008CE08093C400E1ECB4
:10030000F0E0808188608083808180618083E2EC7E
:10031000F0E080818660808308959091C00095FF11
:10032000FCCF8093C60008958091C00087FFFCCF6A
:100330008091C6000895CF93DF93AC01DC0190E07B
:1003400020E03D91FB01E90FF11D8081381320C0B1
:1003500090E0892F820FFA01E80FF11D3081C92F3B
:10036000D0E031110BC0FB0101900020E9F731977B
:10037000E61BF70BCE17DF0759F40FC0FB01EC0F9C
:10038000FD1F8081882379F33813EDCF9F5FE1CF84
:100390002F5F2035B1F680E001C081E0DF91CF9181
:1003A0000895CF93DF93EC018991882319F00E947F
:1003B0008D01FACFDF91CF910895CF93DF93EC01B8
:1003C000CE01FE012491222331F02196FC0184917B
:1003D0000E948D01F5CFDF91CF910895CF931092B8
:1003E000C201C0E50E949401282F30E02A30310577
:1003F00079F02D30310561F0E091C201F0E0EA5B67
:10040000FE4F80838091C2018F5F8093C2010DC037
:100410008091C201882349F0E091C201F0E0EA5BDB
:10042000FE4F10821092C20102C0C150D9F681E085
:10043000CF910895CF931092BF011092C0011092F6
:10044000C201C0E00E949401CF5F8C3219F0C43128
:10045000C9F75EC0C43109F45BC00E949401E09109
:10046000BF01F0E0E65FFE4F80839091BF019F5F88
:100470009093BF01CF5F8C3249F4E091BF01F0E06F
:10048000E75FFE4F10821092BF0105C0C63429F706
:10049000F4CFC63480F40E949401E091C001F0E0F2
:1004A000E25EFE4F80839091C0019F5F9093C001F8
:1004B000CF5F8C3271F7E091C001F0E0E35EFE4F58
:1004C00010821092C00105C02A303105A9F0C6344F
:1004D00098F40E949401282F30E0E091C201F0E0EE
:1004E000EA5BFE4F80838091C2018F5F8093C201DF
:1004F000CF5F2D30310541F7E091C201F0E0EB5BB9
:10050000FE4F10821092C2010E94940181E001C04E
:1005100080E0CF910895CF931092C101C0E00E9476
:100520009401CF5F8A3311F0C035C9F70E9494015E
:10053000CF5F823211F0C035C8F30E949401E09180
:10054000C101F0E0EE5CFE4F80839091C1019F5F9E
:100550009093C101CF5F823249F4E091C101F0E094
:10056000EF5CFE4F10821092C10107C0C03528F326
:10057000F4CF0D9749F0C03538F40E94940190E013
:10058000CF5F8A309105A9F781E0CF910895CF938D
:1005900010929601C0E00E949401CF5F8C3211F05E
:1005A000C634C9F70E949401CF5F8C3211F0C63473
:1005B000C8F30E949401282F30E0E0919601F0E00A
:1005C000E050FF4F8083809196018F5F809396016A
:1005D000CF5F2A30310529F02D30310511F0C634B6
:1005E00040F3E0919601F0E0E150FF4F108210924D
:1005F000960181E0CF910895882361F026E033E1F0
:100600004EEA4A95F1F73A95E1F72A95D1F700C0FD
:100610008150F2CF0895611571058105910549F06A
:1006200020E12A95F1F700C0615071098109910913
:10063000F2CF0895CF938AEA92E00E94DD010E94F2
:10064000EE01882389F043E050E067EA72E087E931
:1006500091E00E94B80567E971E086E491E00E94AC
:100660009B01C1E0813009F0C0E081E00E94FC0202
:10067000CC2309F387E492E00E94DD0181E00E942F
:10068000FC0281E0CF910895CF9382E00E94FC02AA
:100690008EE492E00E94DD010E94EE018823A9F31E
:1006A0004DE050E068E672E087E991E00E94B8050D
:1006B00067E971E086E491E00E949B01C82F4FE05A
:1006C00050E069E572E087E991E00E94B80567E9CA
:1006D00071E086E491E00E949B01813049F40E9420
:1006E000FC0286E392E00E94DD0181E00E94FC02B0
:1006F000C13059F681E0CF910895CF93DF9381E027
:100700000E94FC0281E892E00E94DD010E94EE015D
:10071000811102C0C0E367C04BE050E067E972E0BE
:1007200087E991E00E94B80567E971E086E491E00D
:100730000E949B01813009F469C04BE050E06CE8F5
:1007400072E087E991E00E94B80567E971E086E40C
:1007500091E00E949B018130E9F658C04BE050E0E7
:1007600067E972E087E991E00E94B80567E971E006
:1007700086E491E00E949B01D82F4BE050E06CE8AA
:1007800072E087E991E00E94B80567E971E086E4CC
:1007900091E00E949B018130C9F1D130B9F181E033
:1007A0000E94FC028CED91E00E94DD0181E00E943C
:1007B000FC0283EC91E00E94DD01DEE18CE30E940B
:1007C000FC02D150D9F78AEA92E00E94DD0181E073
:1007D0000E94FC0286EB91E00E94DD0181E00E9414
:1007E000FC02C15099F081E00E94FC0280ED91E092
:1007F0000E94DD0188E70E94FC0281E892E00E94ED
:10080000DD010E94EE01882361F3A8CF81E0DF9132
:10081000CF91089581E00E94FC028EE191E00E9458
:10082000DD0181E00E94FC028EEF90E00E94DD017C
:1008300081E00E94FC028DED90E00E94DD0181E0EC
:100840000E94FC028DEB90E00E94DD0181E00E949D
:10085000FC0281E0089583B7817F846083BF83B702
:10086000816083BF52985A9AF894E9E6F0E080815B
:100870008D7F808380818E7F8083E89A78948895AD
:1008800083B78E7F83BF08951F920F920FB60F928A
:100890001124E8980F900FBE0F901F9018950E949A
:1008A000770152985A9A8AE00E94FC020E941A0329
:1008B00082E00E94FC0288EA91E00E94DD0181E072
:1008C0000E94FC0289E292E00E94DD0181E00E9428
:1008D000FC0285E792E00E94DD0181E00E94FC02BB
:1008E00081EA91E00E94DD0183E00E94FC020E9407
:1008F000440381E00E94FC0280ED91E00E94DD0152
:1009000088E70E94FC020E947D030E940A0487E19E
:1009100092E00E94DD0181E00E94FC0288EF91E0FC
:100920000E94DD0182E00E94FC0288EE91E00E94BC
:10093000DD0181E00E94FC0280E991E00E94DD017E
:1009400081E00E94FC0283EC91E00E94DD0182E0E4
:100950000E94FC0280E8C82E88EAD82E82E1E82EA8
:10096000FF24F3944A9B1AC061E070E080E090E0BD
:100970000E940B0381E0C81AD108E108F10891F741
:100980008AEA92E00E94DD0181E00E94FC0286EB8F
:1009900091E00E94DD010E947D03D2CF0E94EE0112
:1009A0008823D9F145E050E062EA72E087E991E0FE
:1009B0000E94B80567E971E086E491E00E949B011E
:1009C0008130C1F40E948B028AEA92E00E94DD012C
:1009D00081E00E94FC0286EB91E00E94DD0181E053
:1009E0000E94FC0283E292E00E94DD0181E00E940D
:1009F000FC0213C08AEA92E00E94DD0181E00E94BD
:100A0000FC0286EB91E00E94DD0181E00E94FC0285
:100A10000E9444030E947D037ACFC3E081E00E94DC
:100A2000FC0280E990E00E94DD0181E00E94FC026E
:100A30000E940A0481E00E94FC028EEA90E00E947B
:100A4000DD018AE00E94FC028FE990E00E94DD0156
:100A50000E94EE01882389F04CE050E064E870E0E9
:100A600087E991E00E94B80567E971E086E491E0CA
:100A70000E949B0191E0813009F090E0C15019F093
:100A8000992361F203C0913009F06EC081E00E94A9
:100A9000FC0288E690E00E94DD010E94C70281E02E
:100AA0000E94FC0281E790E00E94DD010E941A0290
:100AB000811104C087E30E94FC024FC081E00E94C4
:100AC000FC0287E192E00E94DD0181E00E94FC02CD
:100AD0008DE092E00E94DD0182E391E00E94D1016D
:100AE00084EF91E00E94DD0181E00E94FC0286E437
:100AF00091E00E94D10187E591E00E94DD018AE04A
:100B000091E00E94D1018CE491E00E94DD018EE130
:100B100091E00E94D1018EE391E00E94DD0180E02E
:100B200091E00E94D1018EE691E00E94DD018EE10C
:100B300091E00E94D1018CE691E00E94DD018AE003
:100B400091E00E94D10189E691E00E94DD0181E0FF
:100B50000E94FC028AE10E948D0185E00E94FC0255
:100B600080E990E00E94DD018AE00E94FC02CFCE85
:100B7000FB01DC0102C005900D9241505040D8F7B6
:060B80000895F894FFCF78
:100B8600313233343536373839303132333435361D
:100B96003738393031323334353637383930313207
:100BA60033343536373839303132333435363738F1
:100BB60039303132333435363738393031323334EF
:100BC60035363738393031323334353637383930CF
:100BD60031323334353637383930313233343536CD
:100BE60037383930313233343536373839303132B7
:100BF60033343536373839303132333435363738A1
:100C0600393031323334353637383930313233349E
:060C160035363738393095
:00000001FF
